:020000040000FA
:040000008A01032846
:0A00060083129813831607309C0044
:100010009D019B018316183085008312051E11284F
:10002000D8291E288207543445344D345034453481
:1000300020343D340034D63443340034421933285C
:100040008316851005110030860083128510051176
:100050003830A1200130A1200330A1200F30A12091
:100060008030A120412883168510051100308600BC
:100070008312851005113830A1200C30A120C0302A
:10008000A120B7204420B528831685100511003023
:1000900086008312851005113830A1200130A1207F
:1000A0000330A1200F30A1208030A1201330852003
:1000B0008316851005110030860083128510051106
:1000C0003830A1200C30A120C030A12042186A286D
:1000D000FA30A62030088600A62031088600A62027
:1000E000C21873207C282E30A6203308A62020308A
:1000F000A6201B30932008002030A6202030A62008
:100100002030A6201B3093200800C4001230C40207
:10011000C40344081220C100C10803199228A62074
:10012000C40A89280800C4001230C402C403440869
:100130001220C100C1080319A028A620C40A9728CC
:10014000080086008510AB20C021080086008514B9
:10015000AB20C021080005150000051108003F185C
:10016000B52846088600A6200800CA211E28CB20F4
:10017000E020E2203321E2202B21CB20E020E220EE
:10018000FE20E2200029C0000029BF00CB2035213D
:100190009821A7210800CE20DB20080083168515B2
:1001A00083128316851183128511BA218316851552
:1001B0008312B12108008519DB28851DDD28080080
:1001C000CC300800BD000830BE00831685158312B0
:1001D0008316851183128511BD0C031CF328831629
:1001E00085158312F7288316851183128511B42192
:1001F000831685158312BE0BE8280800BE30080060
:100200000830B500B6018316851583128316851153
:10021000831285110000831685158312AC2103100B
:1002200085190314B60CB421831685158312B50BFA
:100230000629360842192029B8004215C215C328DC
:10024000C219292938020319B5283608B800C21581
:10025000C328C211C528831685158312851D2E2932
:10026000CA2100000800443008003B214E215821DB
:100270007F2193210800C3010330BE000314BF0C8B
:10028000C00CC30CBE0B3E290310C00CC30C0430C1
:10029000BE000310C30CBE0B492908004210031115
:1002A000FF303F0503195629421408004210080088
:1002B00003110030430403197B290C304305031953
:1002C0006F29C3196629431D6B29692943196D29B3
:1002D0006B2972217D2975217D2978217D29313075
:1002E000B30008003330B30008003530B300080015
:1002F0003830B3000800C2100800C21408004008DB
:10030000C501C601C7000A304702031C9029C70077
:10031000C60A0A304602031C8329C601C50A83297E
:10032000460E470708003030C504C604C70408005D
:1003300042189B29FA304608B0004708B100C2189D
:10034000A229A429330808003030B30008002E3059
:10035000B20008000530BC290230BC29033000007F
:10036000BC2905300000BC290F30BC291330BC2942
:100370001630BC29A630BC29BA00BA0BBD2908002A
:100380004030C229BC00FF30BA00BA0BC529BC0BF3
:10039000C32908000630CC29BC00D930BB00FF308F
:1003A000BA00BA0BD129BB0BCF29BC0BCD29080051
:1003B0008501860104308A000030A50083160313EE
:1003C00086008500831203130F22EA21F7210322FE
:1003D0004022E529303084001030A400240825078D
:1003E00043228000840AA40BEE29A50A080080306D
:1003F00018220830A3003F30840000082422840320
:10040000A30BFD290800C03018220830A3003730A4
:100410008400000824228403A30B092A0800383032
:10042000182201301822033018220F301822080039
:1004300086003022043085003022003085003022D2
:100440000430850030220800860030220630850006
:10045000302202308500302206308500302208002C
:100460000A30A200A100A10B332AA20B322A0800F5
:10047000FA30A200A100A10B3B2AA20B3A2A0800E5
:08048000382238220800820036
:100800002E34453456344F344C34553450344934F6
:100810004334203442346F346F3474346C346F3466
:1008200061346434653472342034313436344634BF
:10083000383438342E342E3434344B3420344D3460
:1008400045344D344F3452344934413420344634E5
:100850004C344134533448342E342E34333436340B
:1008600038342034423459345434453453342034E9
:10087000523441344D342E342E34323435343634FF
:1008800020344434453420344534453450345234D3
:100890004F344D342E342E34503455344534523484
:1008A00054344F345334203450344134523441346E
:1008B00020344C34433444342034593420345434B8
:1008C000453443344C34413444344F342E342E3484
:1008D000523445344C3445345634413444344F3426
:1008E00052342034443445342034313432343734B3
:1008F00076342E3420343134203461346D34703405
:100900002E342E34383420344C344534443453346B
:100910002E342E34343420344D344934433452345C
:100920004F345334573449345434433448344534C1
:1009300053342E342E34503452344F3447345234DE
:1009400041344D34413444344F34523420344434EF
:1009500045344C3420343134363446343834383429
:10096000203449344E3454344534473452344134BD
:1009700044344F342E342E34533445344E345334AF
:100980004F345234203444344534203454344534C4
:100990004D34503445345234413454345534523447
:1009A00041342E342E34503455344534523454347A
:1009B0004F342034533445345234493441344C3468
:1009C0002034523453343234333432342E342E34CF
:1009D0004634493452344D3457344134523445341A
:1009E000203442344F344F3454344C344F34413437
:1009F0004434453452342E342E342E342E342E3496
:040A00002E342E342E
:00000001FF
